:020000040000FA
:0A0000000000000093EF00F0ACD008
:08001800FFD09EA8FED7AD6EDB
:100020001200106E960E076E980E086E55D8D8B452
:10003000CA90D8A4CA80FC0FD8A0CA92D8B0CA82ED
:10004000800E076E960E086E980E0B6E0C6ACAB084
:1000500025D8CAB223D842D80704CB6E07C009F00E
:1000600008C00AF002500D6E0E6E023C0E6A4BD8AC
:100070000C50102E0AD0BE6E0C0EBD6E0BBEBD8A8B
:100080000BBCBD889494CA841200BB6E0C0EBA6E71
:100090000BBEBA8A0BBCBA889492F5D700D8D89018
:1000A0000B320832073212000A6A096EFF0E092667
:1000B0000A2200D0D8A01200030E086EE60E02D865
:1000C000F5D7086AFE0F076EE86A085AD8A0120032
:1000D0000000070600D0F8D70C6A0B6A100EF36E0A
:1000E00008340B360C3609500B5C0A500C5805E3EB
:1000F00009500B5E0A500C5AD88007360836F32E8A
:10010000EFD70750120009500D02F3CF0BF0F4CFD8
:100110000CF00A500D02F3500C2609500E02F35059
:100120000C260B501200006A4F0EAF6EB06A240E00
:10013000AC6E900EAB6E00010F0EC16E070EB46E6A
:100140000FEE7EF0ED6AE950EA10FCE1EF6AC69A24
:10015000C30E926EE00E936EC00E946E92809282E9
:1001600070D0F2A409D0F294164A172AD6CF14F010
:10017000D7CF15F0817A11009EAA19D0060EAB14C4
:1001800012E1E2CF30F0E1CF2FF0312A10EE3DF056
:100190003150E126000EE222AECFE7FF30C0E2FF91
:1001A0002FC0E1FF1100AE50AE50AB98AB881100EC
:1001B0003150325C14E0322AEACF08F0E9CF07F080
:1001C00000EE3DF03250E926000EEA22EF502E6E8E
:1001D00008C0EAFF07C0E9FFD880120004D0E86831
:1001E0002E6ED8A012001200316A326A9D8A9F8A50
:1001F000F28EF28C12009D9A00EE3DF0010EF46E2C
:10020000F36AF306000EF45AEE6AF450F310F9E1C3
:10021000316A326A9D8A1200F29EE0CFC1F5D8CFD2
:10022000C2F5E8CFC3F5F28E0001A192B36AB26ABB
:10023000F29EC1C5E0FFC2C5D8FFC3C5E8FFF28E7C
:100240001000939A8A8A0A0E2FDF939A8A9A9298BC
:10025000899893948A94929A899A94908B90949284
:100260008B9294948B9494968B9694988B98949A62
:100270008B9A00EE35F0080EEE68E82EFDD7276A5F
:1002800004EEBDF0010EF46EF36AF306000EF45AAC
:10029000EE6AF450F310F9E1336A346A0501C0697B
:1002A000A3DF0001A8DFCD6AF294F28A870ED56E33
:1002B000B16AA192A082B36AB26AD08EA292B10E44
:1002C000B16E44EC05F045EC09F044EC0BF0D6CFF0
:1002D00014F0D7CF15F06CDF2EC018F0EE0E185CBE
:1002E00006E3FE0E185C01E301D01A6AE1D118AEF4
:1002F00037D01A6A8D0E185C05E118C01AF01B6819
:100300001C682DD09D0E185C05E118C01AF01D6800
:100310001E6825D0AD0E185C05E118C01AF01F68E4
:1003200020681DD0BD0E185C05E118C01AF02168C8
:10033000226815D0CD0E185C04E118C01AF02368AD
:100340000ED0DD0E185C04E118C01AF0246807D046
:10035000ED0E185C04E118C01AF025682668A7D1D4
:100360001A5202E1A5D1A3D18D0E1A5C32E11B28ED
:1003700003E118C01BF02BD018C01CF01B50050166
:10038000BD5D000121E18D0E48DE1B5046DE1C5094
:1003900044DE0501BD6BFF0E1424036EFF0E152015
:1003A000046E000E1620056E000E1720066E06C0A5
:1003B00038F005C037F004C036F003C035F01BC07C
:1003C000BEF5C069000101D073D11B6870D170D136
:1003D0006ED19D0E1A5CD8A42AD11D2803E118C045
:1003E0001DF023D118C01EF01E5229E11D50050139
:1003F000BD5D000121E19D0E10DE1D500EDE000EE0
:100400000CDE0501BD6BFF0E1424036EFF0E1520DC
:10041000046E000E1620056E000E1720066E06C034
:1004200038F005C037F004C036F003C035F01DC009
:10043000BEF5C069000101D03BD139D1F6D027A06B
:10044000F2D0300E1D5CD8A074D03C0E1D5CD8B02C
:1004500070D01D500501BE5D000130E0332A04EE6E
:10046000BDF03350E926000EEA229D0EEF6E332ACE
:1004700004EEBDF03350E926000EEA221DC0EFFF66
:10048000332A04EEBDF03350E926000EEA221EC0E6
:10049000EFFFFA0E1424036E000E1520046E000EFA
:1004A0001620056E000E1720066E06C03CF005C033
:1004B0003BF004C03AF003C039F00BD09D0E0DECB8
:1004C00000F01D500DEC00F01E500DEC00F01DC0B2
:1004D000BDF5386837683668356804EE3DF01D5064
:1004E000EB50286E28B002D08B9801D08B8828B2B0
:1004F00002D08B9001D08B8028B402D08B9A01D08F
:100500008B8A28B602D0899A01D0898A28B802D06D
:100510008B9401D08B8428BA02D08B9601D08B8625
:100520000268520E0A6E080E096E020E11EC00F0FF
:100530007AD03C0E1D5CD8A074D06A0E1D5CD8B079
:1005400070D01D500501BE5D000130E0332A04EE7D
:10055000BDF03350E926000EEA229D0EEF6E332ADD
:1005600004EEBDF03350E926000EEA221DC0EFFF75
:10057000332A04EEBDF03350E926000EEA221EC0F5
:10058000EFFFFA0E1424036E000E1520046E000E09
:100590001620056E000E1720066E06C03CF005C042
:1005A0003BF004C03AF003C039F00BD09D0E0DECC7
:1005B00000F01D500DEC00F01E500DEC00F01DC0C1
:1005C000BDF5386837683668356804EE3DF01D5073
:1005D000EB50286E28B002D08B9801D08B8828B2BF
:1005E00002D08B9001D08B8028B402D08B9A01D09E
:1005F0008B8A28B602D0899A01D0898A28B802D07D
:100600008B9401D08B8428BA02D08B9601D08B8634
:10061000026A520E0A6E080E096E020E11EC00F00C
:1006200002D01D6845D01D6842D042D040D0AD0EEA
:100630001A5C0AE11F2803E118C01FF003D018C09C
:1006400020F0F0D835D033D0BD0E1A5C0AE1212855
:1006500003E118C021F003D018C022F03AD928D005
:1006600026D0CD0E1A5C0DE1232809E118C023F035
:10067000CD0E0DEC00F023500DEC00F0236818D0E7
:1006800016D0DD0E1A5C07E1242803E118C024F01F
:100690001ED90ED00CD0ED0E1A5C09E1252803E11D
:1006A00018C025F003D018C026F0D4D801D080D8C7
:1006B000020E2D5CD8B073D02950145C2A50155806
:1006C0002B5016582C501758D8A05CD02C8E2D5279
:1006D00017E18B988B9A899A8B908B948B96026AF0
:1006E000520E0A6E080E096E020E11EC00F0286A16
:1006F00038683768366835680501BE6B000141D03F
:10070000010E2D5C3EE1342A04EEBDF03450E926A2
:10071000000EEA22EF500DEC00F004EEBDF0345074
:10072000E926000EEA22EF500501BF6F342A04EEDD
:10073000BDF03450E926000EEA22EF500DEC00F037
:100740009D0E0501BF5D000109E104EEBDF03450CE
:10075000E926000EEA22EF500501BD6F0001342AA0
:1007600004EEBDF03450E926000EEA22EF500DEC05
:1007700000F03C683B683A6839683350345C01E00B
:10078000C2D716D817AE0AD0176A166A156A146A45
:1007900000EE35F0080EEE68E82EFDD706D017AE55
:1007A00004D0176A166A156A146A817067EF01F03F
:1007B0002D682C8E196A020E195C33E2D890193418
:1007C000E96EEA6AEA36E936EA36350EE926000EBF
:1007D000EA22EFCF03F0ECCF04F0ECCF05F0ECCF42
:1007E00006F02950035C2A5004582B5005582C5011
:1007F000065815E2D8901934E96EEA6AEA36E93605
:10080000EA36350EE926000EEA22EFCF29F0ECCFCA
:100810002AF0ECCF2BF0ECCF2CF019C02DF0192AD8
:10082000CAE31200300E1F5C11E36A0E1F5C0EE279
:10083000300E0501BD5D000109E3AD0E0DEC00F0C9
:100840001F500DEC00F020500DEC00F01F6812005E
:1008500023681200300E0501BD5D000111E3265032
:100860000501C05D00010BE0ED0E0DEC00F0255020
:100870000DEC00F026500DEC00F026C0C0F525D0A0
:1008800026500501C05D000120E03350345C1DE0BE
:10089000332A04EEBDF03350E926000EEA22ED0EB5
:1008A000EF6E332A04EEBDF03350E926000EEA2243
:1008B00025C0EFFF332A04EEBDF03350E926000EC9
:1008C000EA2226C0EFFF26C0C0F525681200246882
:1008D0001200010E215C0AE1BD0E0DEC00F0010ECC
:1008E0000DEC00F022500DEC00F0B4D0020E215CB3
:1008F0003FE1300E0501BD5D000109E2026A520EC2
:100900000A6E080E096E020E11EC00F030D0300EA7
:100910000501BD5D00010EE33C0E0501BD5D00015A
:1009200009E20268520E0A6E080E096E020E11EC00
:1009300000F01DD03C0E0501BD5D000110E36A0E04
:100940000501BD5D00010BE222502224026E520E11
:100950000A6E080E096E020E11EC00F008D0026A51
:10096000520E0A6E080E096E020E11EC00F072D0E3
:10097000030E215C0DE3080E215C0AE2BD0E0DECB6
:1009800000F021500DEC00F022500DEC00F062D090
:100990000F0E215C0DE3150E215C0AE2BD0E0DEC7D
:1009A00000F021500DEC00F022500DEC00F052D080
:1009B000420E215C13E1BD0E0DEC00F0420E0DEC79
:1009C00000F022500DEC00F0225203E1279044D8B1
:1009D00004D0929889888A8427803CD0500E215C6C
:1009E0000AE1BD0E0DEC00F021500DEC00F022509C
:1009F0000DEC00F02FD0640E215C0DE3700E215C35
:100A00000AE2BD0E0DEC00F021500DEC00F022507A
:100A10000DEC00F01FD07B0E215C1BE1BD0E0DEC38
:100A200000F07B0E0DEC00F0000E0DEC00F0899A4A
:100A30008B908B968B988B9A8B94026A520E0A6ECF
:100A4000080E096E020E11EC00F0286A0501BE6B5B
:100A5000C06B000121681200929889988A94899A43
:100A60008B90026A520E0A6E080E096E020E11EC8D
:100A700000F08B968B988B9A8B94286A276A0501D5
:100A8000BE6BC06B0001120002013E693D695C0E45
:100A9000406F7A0E3F6F590E426F850E416F580EB0
:100AA000446F140E436F560E466FA90E456F550ED8
:100AB000486F430E476F530E4A6FE30E496F520E55
:100AC0004C6F890E4B6F510E4E6F350E4D6F4F0EA2
:100AD000506FE60E4F6F4E0E526F9C0E516F4D0EC3
:100AE000546F580E536F4C0E566F190E556F4A0EB9
:100AF000586FDF0E576F490E5A6FAA0E596F480E86
:100B00005C6F7A0E5B6F470E5E6F4F0E5D6F460E29
:100B1000606F290E5F6F450E626F080E616F430EA6
:100B2000646FEB0E636F420E666FD30E656F410EFE
:100B3000686FBF0E676F400E6A6FB00E696F3F0E31
:100B40006C6FA50E6B6F3E0E6E6F9E0E6D6F3D0E41
:100B5000706F9C0E6F6F3C0E726F9E0E716F3B0E2E
:100B6000746FA40E736F3A0E766FAE0E756F390EFA
:100B7000786FBC0E776F380E7A6FCE0E796F370EA6
:100B80007C6FE30E7B6F360E7E6FFD0E7D6F360E33
:100B9000806F1A0E7F6F350E826F3B0E816F340EA1
:100BA000846F5F0E836F330E866F870E856F320EF4
:100BB000886FB20E876F310E8A6FE10E896F310E2A
:100BC0008C6F140E8B6F300E8E6F490E8D6F2F0E43
:100BD000906F820E8F6F2E0E926FBE0E916F2D0E44
:100BE000946FFD0E936F2D0E966F3F0E956F2C0E2A
:100BF000986F850E976F2B0E9A6FCD0E996F2B0EF7
:100C00009C6F180E9B6F2A0E9E6F670E9D6F290EAC
:100C1000A06FB80E9F6F290EA26F0C0EA16F280E49
:100C2000A46F620EA36F270EA66FBC0EA56F270ED2
:100C3000A86F180EA76F260EAA6F760EA96F250E45
:100C4000AC6FD80EAB6F250EAE6F3C0EAD6F240EA1
:100C5000B06FA20EAF6F240EB26F0B0EB16F230EEA
:100C6000B46F760EB36F220EB66FE40EB56F220E20
:100C7000B86F540EB76F210EBA6FC60EB96F210E42
:100C8000BC6F3B0EBB6F200EBE6FB20EBD6F200E51
:100C9000C06F2B0EBF6F1F0EC26FA60EC16F1F0E4F
:100CA000C46F240EC36F1E0EC66FA30EC56F1E0E3B
:100CB000C86F250EC76F1D0ECA6FA90EC96F1D0E16
:100CC000CC6F2E0ECB6F1C0ECE6FB60ECD6F1C0EE2
:100CD000D06F3F0ECF6F1B0ED26FCB0ED16F1B0E9E
:100CE000D46F580ED36F1A0ED66FE80ED56F1A0E4A
:100CF000D86F790ED76F1A0EDA6F0B0ED96F190EE7
:100D0000DC6FA00EDB6F190EDE6F360EDD6F180E76
:100D1000E06FCE0EDF6F180EE26F680EE16F180EF7
:100D2000E46F030EE36F170EE66FA00EE56F170E6C
:100D3000E86F3F0EE76F160EEA6FDF0EE96F160ED3
:100D4000EC6F800EEB6F160EEE6F240EED6F150E2E
:100D5000F06FC80EEF6F150EF26F6E0EF16F150E7D
:100D6000F46F160EF36F140EF66FBF0EF56F140EC0
:100D7000F86F690EF76F140EFA6F150EF96F130EF8
:100D8000FC6FC20EFB6F130EFE6F710EFD6F130E24
:100D90000301006F210E0201FF6F120E0301026FAB
:100DA000D20E016F120E046F840E036F120E066FC7
:100DB000380E056F110E086FED0E076F110E0A6FDA
:100DC000A30E096F110E0C6F5A0E0B6F110E0E6FE2
:100DD000120E0D6F100E106FCC0E0F6F100E126FE3
:100DE000870E116F100E146F420E136F0F0E166FD9
:100DF0001569186FBD0E176F0F0E1A6F7C0E196FE5
:100E00000F0E1C6F3D0E1B6F0E0E1E6FFE0E1D6F24
:100E10000E0E206FC00E1F6F0E0E226F830E216FFD
:100E20000E0E246F470E236F0E0E266F0C0E256FCD
:100E30000D0E286FD20E276F0D0E2A6F990E296F97
:100E40000D0E2C6F610E2B6F0D0E2E6F2A0E2D6F57
:100E50000C0E306FF40E2F6F0C0E326FBE0E316F12
:100E60000C0E346F8A0E336F0C0E366F560E356FC4
:100E70000C0E386F230E376F0B0E3A6FF10E396F71
:100E80000B0E3C6FC00E3B6F3E693D69A20E406F7A
:100E9000C30E3F6F9A0E426F460E416F960E446F1F
:100EA000320E436F920E466F3A0E456F8E0E486FAC
:100EB0005D0E476F8A0E4A6F9A0E496F860E4C6F11
:100EC000F00E4B6F830E4E6F5F0E4D6F7F0E506FA7
:100ED000E70E4F6F7C0E526F850E516F790E546F77
:100EE0003B0E536F760E566F070E556F720E586F8E
:100EF000E80E576F6F0E5A6FDF0E596F6C0E5C6FF6
:100F0000EA0E5B6F6A0E5E6F0A0E5D6F670E606FB2
:100F10003C0E5F6F640E626F820E616F610E646FD4
:100F2000DA0E636F5F0E666F440E656F5C0E686F5E
:100F3000BF0E676F5A0E6A6F4C0E696F570E6C6F5B
:100F4000E90E6B6F550E6E6F960E6D6F530E706FD0
:100F50006F6F510E726F200E716F4E0E746FFB0E1D
:100F6000736F4C0E766FE50E756F4A0E786FDC0E60
:100F7000776F480E7A6FE20E796F460E7C6FF50E32
:100F80007B6F450E7E6F150E7D6F430E806F420E98
:100F90007F6F410E826F7B0E816F3F0E846FC00E9C
:100FA000836F3E0E866F100E856F3C0E886F6D0E40
:100FB000876F3A0E8A6FD40E896F390E8C6F460E8A
:100FC0008B6F370E8E6FC20E8D6F360E906F490E7F
:100FD0008F6F340E926FDA0E916F330E946F740E22
:100FE000936F320E966F180E956F300E986FC50E78
:100FF000976F2F0E9A6F7B0E996F2E0E9C6F3A0E85
:101000009B6F2D0E9E6F020E9D6F2B0EA06FD10E4B
:101010009F6F2A0EA26FA90EA16F290EA46F880ED2
:10102000A36F280EA66F6F0EA56F270EA86F5E0E1A
:10103000A76F260EAA6F530EA96F250EAC6F500E28
:10104000AB6F240EAE6F540EAD6F230EB06F5E0EFD
:10105000AF6F220EB26F6F0EB16F210EB46F860E9E
:10106000B36F200EB66FA30EB56F1F0EB86FC60E0E
:10107000B76F1E0EBA6FEF0EB96F1E0EBC6FBB6F4F
:101080001D0EBE6F520EBD6F1C0EC06F8C0EBF6F5B
:101090001B0EC26FCB0EC16F1B0EC46F0F0EC36F42
:1010A0001A0EC66F580EC56F190EC86FA50EC76F02
:1010B000180ECA6FF80EC96F180ECC6F4F0ECB6F9B
:1010C000170ECE6FAB0ECD6F170ED06F0A0ECF6F0F
:1010D000160ED26F6F0ED16F150ED46FD70ED36F61
:1010E000150ED66F430ED56F140ED86FB30ED76F93
:1010F000140EDA6F270ED96F130EDC6F9F0EDB6FA5
:10110000130EDE6F1A0EDD6F120EE06F990EDF6F99
:10111000120EE26F1B0EE16F110EE46FA10EE36F72
:10112000110EE66F290EE56F100EE86FB50EE76F32
:10113000100EEA6F440EE96F0F0EEC6FD60EEB6FD8
:101140000F0EEE6F6B0EED6F0F0EF06F030EEF6F65
:101150000E0EF26F9D0EF16F0E0EF46F3A0EF36FDE
:101160000D0EF66FDA0EF56F0D0EF86F7C0EF76F41
:101170000D0EFA6F210EF96F0C0EFC6FC80EFB6F8F
:101180000C0EFE6F720EFD6F0C0E0401006F1E0E32
:101190000301FF6F0B0E0401026FCC0E016F0B0EEB
:1011A000046F7C0E036F0B0E066F2E0E056F0A0E7A
:1011B000086FE30E076F0A0E0A6F990E096F0A0E89
:1011C0000C6F510E0B6F0A0E0E6F0B0E0D6F090E8A
:1011D000106FC80E0F6F090E126F850E116F090E7A
:1011E000146F450E136F090E166F060E156F080E5D
:1011F000186FC90E176F080E1A6F8E0E196F080E32
:101200001C6F540E1B6F080E1E6F1C0E1D6F070EF9
:10121000206FE50E1F6F070E226FAF0E216F070EB6
:10122000246F7B0E236F070E266F490E256F070E66
:10123000286F170E276F060E2A6FE70E296F060E0E
:101240002C6FB90E2B6F060E2E6F8B0E2D6F060EA8
:10125000306F5F0E2F6F060E326F340E316F060E39
:10126000346F0A0E336F050E366FE10E356F050EC3
:10127000386FB90E376F050E3A6F930E396F050E42
:101280003C6F6D0E3B6F00011200040E0101406FB8
:10129000880E3F6F040E426FA60E416F040E446F1E
:1012A000B60E436F040E466FC60E456F040E486FB0
:1012B000D60E476F040E4A6FE60E496F040E4C6F50
:1012C000F60E4B6F050E4E6F070E4D6F050E506FED
:1012D000170E4F6F050E526F280E516F050E546F8B
:1012E000390E536F050E566F4B0E556F050E586F26
:1012F0005D0E576F050E5A6F6E0E596F050E5C6FBF
:10130000800E5B6F050E5E6F930E5D6F050E606F56
:10131000A50E5F6F050E626FB80E616F050E646FEC
:10132000CB0E636F050E666FDF0E656F050E686F7F
:10133000F20E676F060E6A6F696F6C6F1A0E6B6F35
:10134000060E6E6F2E0E6D6F060E706F430E6F6F72
:10135000060E726F580E716F060E746F6D0E736FFE
:10136000060E766F830E756F060E786F980E776F88
:10137000060E7A6FAE0E796F060E7C6FC40E7B6F11
:10138000060E7E6FDB0E7D6F060E806FF20E7F6F96
:10139000070E826F090E816F070E846F210E836F17
:1013A000070E866F380E856F070E886F500E876F99
:1013B000070E8A6F690E896F070E8C6F810E8B6F17
:1013C000070E8E6F9A0E8D6F070E906FB40E8F6F93
:1013D000070E926FCD0E916F070E946FE70E936F0D
:1013E000080E966F020E956F080E986F1D0E976F80
:1013F000080E9A6F380E996F080E9C6F530E9B6FF4
:10140000080E9E6F6F0E9D6F080EA06F8B0E9F6F64
:10141000080EA26FA70EA16F080EA46FC40EA36FD3
:10142000080EA66FE10EA56F080EA86FA769090E3A
:10143000AA6F1D0EA96F090EAC6F3B0EAB6F090EA4
:10144000AE6F5A0EAD6F090EB06F790EAF6F090E09
:10145000B26F990EB16F090EB46FB90EB36F090E6A
:10146000B66FD90EB56F090EB86FFA0EB76F0A0EC8
:10147000BA6F1B0EB96F0A0EBC6F3D0EBB6F0A0E22
:10148000BE6F5F0EBD6F0A0EC06F820EBF6F0A0E79
:10149000C26FA50EC16F0A0EC46FC80EC36F0A0ECD
:1014A000C66FEC0EC56F0B0EC86F110EC76F0B0E1B
:1014B000CA6F360EC96F0B0ECC6F5B0ECB6F0B0E67
:1014C000CE6F810ECD6F0B0ED06FA70ECF6F0B0EB0
:1014D000D26FCE0ED16F0B0ED46FF50ED36F0C0EF4
:1014E000D66F1D0ED56F0C0ED86F460ED76F0C0E33
:1014F000DA6F6F0ED96F0C0EDC6F980EDB6F0C0E6F
:10150000DE6FC20EDD6F0C0EE06FED0EDF6F0D0EA5
:10151000E26F180EE16F0D0EE46F430EE36F0D0ED8
:10152000E66F700EE56F0D0EE86F9C0EE76F0D0E07
:10153000EA6FCA0EE96F0D0EEC6FF80EEB6F0E0E30
:10154000EE6F260EED6F0E0EF06F550EEF6F0E0E56
:10155000F26F850EF16F0E0EF46FB60EF36F0E0E76
:10156000F66FE70EF56F0F0EF86F180EF76F0F0E90
:10157000FA6F4B0EF96F0F0EFC6F7E0EFB6F0F0EA6
:10158000FE6FB10EFD6F0F0E0201006FE60E01013E
:10159000FF6F100E0201026F1B0E016F100E046F21
:1015A000500E036F100E066F870E056F100E086F3A
:1015B000BE0E076F100E0A6FF60E096F110E0C6F3C
:1015C0002E0E0B6F110E0E6F680E0D6F110E106F39
:1015D000A20E0F6F110E126FDC0E116F120E146F30
:1015E000180E136F120E166F540E156F120E186F21
:1015F000910E176F120E1A6FCF0E196F130E1C6F0C
:101600000E0E1B6F130E1E6F4D0E1D6F130E206FEF
:101610008E0E1F6F130E226FCF0E216F140E246FCC
:10162000110E236F140E266F540E256F140E286FA3
:10163000980E276F140E2A6FDC0E296F150E2C6F73
:10164000220E2B6F150E2E6F680E2D6F150E306F3C
:10165000B00E2F6F150E326FF80E316F160E346FFD
:10166000410E336F160E366F8C0E356F160E386FB7
:10167000D70E376F170E3A6F230E396F170E3C6F68
:10168000700E3B6F00011200350E04016D6F340EB9
:101690006E6F6F6F360E706F716F726F320E736F89
:1016A0003A0E746F756F320E766F776F220E786F09
:1016B0006DC403F003C079F46EC403F003C07AF480
:1016C0006FC403F003C07BF470C403F003C07CF468
:1016D00071C403F003C07DF472C403F003C07EF450
:1016E00073C403F003C07FF474C403F003C080F438
:1016F00075C403F003C081F476C403F003C082F420
:1017000077C403F003C083F478C403F003C084F407
:10171000020E856F866F340E876F360E886F896F65
:101720008A6F320E8B6F8C6F3A0E8D6F320E8E6F0A
:10173000260E8F6F220E906F020E916F926F320EF7
:10174000936F3E0E946F3A0E956F360E966F320E73
:10175000976F120E986F1A0E996F360E9A6F340E9D
:101760009B6F300E9C6F1C0E9D6F020E9E6F320E93
:101770009F6F3E0EA06F3A0EA16F360EA26F320E13
:10178000A36F120EA46F1A0EA56F360EA66F00017E
:0617900012001200FFD759
:020000040030CA
:0300010006160ED2
:020005008580F4
:060008000FC00FE00F40E5
:00000001FF
